:020000020000FC
:0200000040C0FE
:1000080000C05FB652B35F7852BB57E058BBDD27DC
:10001800C0980000809BDF5F58BBC1980000809BA0
:10002800DE5F58BBC2980000809BDC5F58BB2395FD
:10003800233009F422272F9358E0550F2A95EAF721
:100048002F911F9312B31F78152B12BBFF27E22F96
:10005800EA5E50811127E6E6F4E0E50FF11FC89546
:1000680008BA223009F4C79A43954A3F11F4442745
:100078003395AA951F915FBE18950FED0DBF0FEF31
:1000880007BB0EEF01BB01E002BB44273327222741
:100098000EE30BBD0FE70ABD09E00EBD00E409BF82
:1000A800789447D169D1B8D1662009F4BF98D03087
:1000B800F1F7A9E1AA23F1F7D63069F0D53061F05C
:1000C800D13039F0D23031F0D33039F0D43031F08A
:1000D800F0CF4AC05FC040C043C03AC0162F170FC8
:1000E800180F09F46EC08ED1F894442733270027DF
:1000F8000DBD0CBD939A78942DD1162F170F180F9C
:1001080009F1D13091F03323C1F3662311F06A95D8
:100118000AC0772319F07A9569E005C08A9569E0E5
:10012800662071F075E03327E8CF9398DD23F1F767
:10013800D23019F0D430C9F2FBCFDD23F1F79DCFCF
:1001480079E0F1CF9398FBD0882009F069C0ABCF54
:1001580081E073E065E0ABCF82E073E060E0A7CFB9
:1001680083E074E060E0A3CF693011F06395A1CF1C
:10017800662029F4793041F0739566279ACF753057
:1001880019F07395662795CF893019F083957727ED
:1001980066278FCF662311F06A958BCF772319F0E6
:1001A8007A9569E086CF662031F4882349F08A95EC
:1001B80079E069E07ECF882319F08A9575E069E0D7
:1001C80078CF4427332700270DBD0CBD939A789428
:1001D800C1D0D130E1F03323E1F33327693011F096
:1001E8006395F7CF662011F4793001C0753019F0A6
:1001F80066277395EECFAED0893021F083957727A7
:100208006627E7CFA7D0882777276627E2CF939876
:10021800D23019F0D430A9F2FBCFDD23F1F72DCF7E
:10022800BF986AE07AE08AE088D060E17AE08AE004
:1002380084D061E170E18AE080D062E171E180E11F
:100248007CD06AE072E181E178D06AE07AE082E10C
:1002580074D060E07AE08AE070D06FE070E08AE005
:100268006CD06FE07FE080E068D06AE07FE08FE0EC
:1002780064D06AE07AE08FE060D06AE07AE08AE0F1
:1002880012D080E018D07FE01ED06FE0AAEF49D0EE
:1002980022D009D080E10FD071E115D062E1AAEF38
:1002A80040D019D0BDCFB4E08AE03AD083E138D04D
:1002B800BA95D1F70895B2E07AE032D073E130D040
:1002C800BA95D1F70895B2E06AE02AD063E128D060
:1002D800BA95D1F708956AE07AE08AE021D094E0EF
:1002E80083951ED09A95E1F794E0739519D09A9565
:1002F800E1F794E0639514D09A95E1F7AAEF11D04D
:1003080094E08A950DD09A95E1F794E07A9508D013
:100318009A95E1F794E06A9503D09A95E1F70895E4
:10032800AEE1D43019F0AA23E1F70895D030F1F7FF
:10033800A4CEA8E2AA23F1F70895ABE4F2CF0AD03D
:10034800EFDF08D0EDDF06D0EBDF04D003D002D01A
:1003580001D00895772079F090E0B0E0BA95B738E9
:10036800E9F79198929ABB27BA95B738E9F7919A25
:1003780092989A9591F70895D03071F0D13069F03C
:10038800D33071F0D23091F0D63099F0D73001F1F6
:10039800D430A9F0D530B1F008957724739401C012
:1003A8007724BF9882E174E1672D1DC08824839467
:1003B80001C08824BF9880E174E1682D14C06624C8
:1003C800639401C06624BF9885E174E1662D0BC073
:1003D80001E0602E802E702E82E071E060E012D085
:1003E8008EE07EE06EE0DD23F1F7BF9A01D008953C
:1003F80004E0172D2AD005E0182D27D006E0162D89
:1004080024D0089501E0162F20D002E0172F1DD028
:1004180003E0182F1AD0089501E011D0612F02E0EF
:100428000ED0712F03E00BD0812F04E008D0712E7D
:1004380005E005D0812E06E002D0612E0895E199ED
:10044800FECF0EBBE09A1DB30895F894E199FECF54
:100458000EBB1DBBF894E29AE19A789408953F0682
:100468005B4F666D7D077F6F000818585C71773E9B
:040478006D08403E8D
:00000001FF
